:10079C002025322E58200025730020537973746560
:1007AC006D2048414C54454400204C6F632E20531F
:1007BC00746570706572206572726F720020537967
:1007CC007374656D20524553455400202E2E2E2EE9
:1007DC00204372656174696E672072616D702000D0
:1007EC00202E2E2E2E2E2046696E652061646A7591
:1007FC0073742020002044652D53796E6368726FEA
:10080C006E697A6564202000496E697420536C69A6
:10081C00646573202E2E2E002020202E2E2E20508C
:10082C006C65617365207761697400204D65636840
:10083C00616E6963616C204572726F7200202020BA
:10084C002E2E2E2053796E6368726F6E697A6564F2
:10085C00002E2E2E4F766572666C6F7720746F208B
:10086C004D494E2020002E2E2E556E646572666CFE
:10087C006F7720746F204D415820002E2E2E41642E
:10088C0076616E636520746F2025342E64002E2EE5
:10089C002E5265766572736520746F2025342E6434
:1008AC0000204D4F5645204572726F7200202E2E3F
:1008BC002E205361766500202E2E2E2045646974FF
:1008CC00002042617365202025332E64202D2030BA
:1008DC0078255820200020536C696465204E756D76
:1008EC0062657220256420002056616C75653A2083
:1008FC0025642073202000204379636C653A202501
:10090C0064207320200020456E61626C65642000B9
:10091C002044697361626C6564002056616C756576
:10092C003A202564205B25255D20200020466F722F
:10093C0077617264202000204261636B776172647E
:10094C007300204C4F4720202D202025322E640090
:10095C0020436F6E6669726D2052454C4F414420A6
:10096C002E2E2E00202E2E2E204C6F6164656400DE
:10097C002045726173652043616C696272617469B0
:10098C006F6E203F00202E2E2E2045726173656401
:10099C00002041646A75737420506F736974696FB9
:1009AC006E0020536C6964652025322E64204465EA
:1009BC00762025322E642000205361766520536505
:1009CC007474696E6773202E2E2E20200020436FC6
:1009DC006E6669726D20434D44202E2E2E002053DE
:1009EC00656C65637420536C69646520312021212A
:1009FC00002056616C75653A202564205B312F31DF
:100A0C0030206D6D5D20200020436F6E6669726D25
:100A1C002054657374202E2E2E00205344785020C1
:100A2C00434F4D4D206572726F72200020534478F5
:100A3C005020434F4D4D2070617373656400204D01
:100A4C004F56454D454E54207061737365642000BC
:100A5C00204D4F56454D454E54206572726F722095
:100A6C002000204465766963652046554E43544901
:100A7C004F4E204F4B202000204465766963652043
:100A8C004D414C46554E4354494F4E202000536F18
:100A9C006674205265736574202E2E2E00202E2E27
:100AAC002E20506C65617365205761697400202E8F
:100ABC002E2E2053656C656374202020202020206E
:100ACC00202000202E2E2E2045646974202000202A
:100ADC002E2E2E2043616E63656C20496E707574EA
:100AEC0000202E2E2E2053656C65637400534C49E8
:100AFC0044452056494557202041524332202F313E
:100B0C00300076657273696F6E20322E3538005066
:100B1C004547415355532039382E2E2E3031002065
:100B2C005344785020434F4D4D206572726F7200C4
:100B3C00494E495420627970617373656400257362
:100B4C00202D2025322E64202F2025322E642000CB
:100B5C002054696D65206C6566743A2025332E64CB
:100B6C00202020200020416E616C6F67205B2525C2
:100B7C005D2025322E642025322E64202000204159
:100B8C0075746F205363726F6C6C696E67002044D0
:100B9C006D782025332E64202D2025332E642025BE
:100BAC00332E6420200000000000000008A000008C
:100BBC00113F000019DF0000227E00002B1E0000F8
:100BCC0033BD00003C5D000044FC00004D9C000067
:100BDC00563B205072696D61727920636F6E74722E
:100BEC006F6C202000002053657175656E7469610F
:100BFC006C2061636365737300002052616E646FD7
:100C0C006D20416363657373202020200000204118
:100C1C0075746F2054696D6572202020202020206F
:100C2C000000205363726F6C6C696E67202020206B
:100C3C002020202000002053696E676C6520202046
:100C4C00202020202020000020556E692D44697240
:100C5C00656374202020202000002042692D446907
:100C6C0072656374202020202020000020556E69BE
:100C7C002D44697265637420496E742E0000204205
:100C8C00692D44697265637420496E742E200000CE
:100C9C004F7065726174696F6E206D6F6465202092
:100CAC000000444D582061646472657373202020E9
:100CBC0020200000536C696465204E756D6265726E
:100CCC002020202000004578706F737572652074A9
:100CDC00696D652020200000466164696E67207490
:100CEC00696D65202020202000004175746F5469C7
:100CFC006D6572204D6F646520200000536875741B
:100D0C0074657220436F6E74726F6C2000005363B5
:100D1C00726F6C6C2073706565642020202000005D
:100D2C005363726F6C6C20646972656374696F6E67
:100D3C00000041636F757374696320626565702090
:100D4C002020000052656C6F6164206465666175DB
:100D5C006C747320000043616C6962726174696F1A
:100D6C006E2020202020000042656C7420636F727E
:100D7C0072656374696F6E2000004572726F722029
:100D8C00636F646520202020202000004469616787
:100D9C006E6F737469637320202020000000507202
:100DAC00696D617279200053657175656E636500BC
:100DBC0052616E646F6D20200054696D6572202045
:100DCC0020005363726F6C6C20200020204E6F202B
:100DDC00726563657074696F6E004E6F2044494D87
:100DEC004D4552206461746100202020446D7820B0
:100DFC0064617461204F4B0013202D394653606C95
:080E0C007986939FACB9C6D2B0
:1032C300C113C115C114C192C116C111C117016245
:0132D30000FA
:05332A00D2F8D2F922E7
:082691008F408B418A4289430E
:10269900C2F8120048C2F9E54025E054FEF540E4CD
:1026A900FFE54025E0F54092F8D2F9C2F90FBF08DD
:1026B900F0D2F8D2F9A2F8B3920AC2F9200902D2EB
:1026C9000A300A41E544603DAB41AA42A9431212CE
:1026D90066FEE4FFEE25E0FE92F8D2F9C2F90FBFDB
:1026E90008F2D2F8D2F9A2F8B3920AC2F974012514
:1026F90043F543E43542F5421544200902D20AD292
:10270900AED2BE80BCC2F8D2F9120048D2F8A20AF1
:01271900229D
:0820DD008F3F8B408A418942CC
:1020E500E4F545754680C2F8120048C2F9E53F257A
:1020F500E04401F53FE4F544E53F25E0F53F92F87E
:10210500D2F9C2F90544E544B408EDD2F8D2F9A2F2
:10211500F8B39208C2F9300850E543604CE4FFF586
:1021250044D2F930F804E5464207C2F9E546C3133F
:10213500F5460544E544B408E8AB40AA41A942EF99
:1021450012127F1543E5436004C2F88002D2F8D22B
:10215500F9120048C2F974012542F542E43541F50A
:10216500410545D2AED2BE80ADC2F8D2F9120048C3
:04217500D2F8AF45A8
:012179002243
:10310600C208753F0A786AA60708A60520081FE5C3
:103116003F601B7F017E001200037B007A00796A04
:10312600754402D2097F50122691920880DEA208C9
:013136002276
:10302D00C205752E0A786AA607ECFF3395E0EF0806
:10303D00F6ED08F620051FE52E601B7F017E0012C0
:10304D0000037B007A00796A754403D2097F501220
:08305D002691920580DEA20518
:013065002248
:1031BC00786AA6077B007A00796A754401D2097F88
:1031CC00501226917B007A00796A7543017F501268
:0731DC0020DD786AE6FF2206
:022D63008F37A8
:102D6500786AA6377B007A00796A754401D2097FB3
:102D7500501226917B007A00796A7543017F5012C3
:102D850020DD786AE6F538E53704F67B007A0079C8
:102D95006A754401D2097F501226917B007A007929
:102DA5006A7543017F501220DDE538FE786AE67CBE
:072DB500002400FFEC3EFECC
:012DBC0022F4
:05332F00D2B4D2B5226A
:042EAA008F3A8D3B93
:102EAE00E53B6030A83AE6F53D753C08E53C601719
:102EBE00E53D25E0F53D153C92B4C2B5D2B57F6433
:102ECE007E0012316780E5053A153B7F647E001265
:102EDE00316780CCD2B4D2B57FF47E011231673027
:052EEE00B402C322D371
:012EF30022BC
:102E5F00752F7820940BA20692087F0A7E001230FD
:102E6F006643E80FD2EED2ECE5E8540FF52E3005AD
:102E7F001D20941AE52F600B7F0A7E0012000315A8
:102E8F002F80EED2087F0A7E0012306680E3C2EEFA
:0A2E9F00C2ECC2C1C213D2B9AF2EBB
:012EA9002206
:1031E300752B7820941AE52B600B7F0A7E00120062
:1031F30003152B80EED2087F0A7E0012306680E32F
:06320300C2C1C213D2B9E2
:0132090022A2
:0D3305003094097F017E0012000380F42245
:022EF4008F3C11
:102EF6007F301231BC8F3DE53D2431FFAD3C1231B0
:102F060006053DE53DC3940550028001C34003E438
:102F1600F53DAD3D7F30123106E4F53ED2087F1E09
:102F26007E001230667FC87E00120003053EE53E35
:052F3600C3940640E712
:012F3B002273
:102DBD007F301231BC8F2C152CE4F52DE52CC394EE
:102DCD000550028001C34003752C04E52C2431FF0E
:102DDD001231BC742E252DF8A607152C052DE52DC9
:102DED00C3940540D7E4F52D7BFF7A07799C742EAB
:102DFD00252DF8E6753F00F540120E76052DE52DD3
:052E0D00C3940540E341
:012E1200229D
:10323000E4FD7F30123106E4F52CE52C2431FF7DCE
:0D324000FF123106052CE52CC3940540ED6E
:01324D00225E
:102FB9008B2C8A2D892E1232857F401232B0852CB6
:102FC9003F852D40852E417BFF7A0779A3120E7626
:102FD9007F141232B07BFF7A0779A6120E767FF240
:0A2FE900122EF4D2AED2BE80FA22FE
:103137001232857F401232B07BFF7A0779B5120EC3
:10314700767F141232B07BFF7A0779C9120E767F29
:10315700F1122EF4D2087FD07E0712306680FE224D
:04271A008F2D8D2E44
:10271E00752F05753005C204786A768008768108B3
:10272E007682796AE718262482786DF6200445E5CC
:10273E00306041E52DC313452EFF7B007A00796A88
:10274E00754404D2091226914011E52F600DD2086E
:10275E007F0A7E00123066152F80D87F907E011280
:10276E00316720F904D20480077F327E0012000305
:10277E00153080B87FC87E00120003E52F6006E595
:10278E00306002D322D2087FD07E0712306612311B
:02279E0037C33F
:0127A0002216
:08233E008F348D358A368B3790
:10234600753805753905C204786A7690E536FF3327
:1023560095E0EF08F6AF37E53708F6FF796AE71834
:10236600262F786DF6200445E5396041E534C31320
:102376004535FF7B007A00796A754404D209122636
:10238600914011E538600DD2087F0A7E0012306652
:10239600153880D87F907E0112316720F904D20467
:1023A60080077F327E00120003153980B87FC87E11
:1023B60000120003E5386009E5396005AE36AF372F
:0823C600221231377EFF7FFF78
:0123CE0022EC
:042A2D008F2F8D302A
:102A3100753305753405C205786A76A008A60308C2
:102A4100A632796AE718262532786DF6200545E524
:102A5100346041E52FC3134530FF7B007A00796A6A
:102A6100754404D2091226914011E533600DD20854
:102A71007F0A7E00123066153380D87F907E011266
:102A8100316720F904D20580077F327E00120003EE
:102A9100153480B87F647E00120003E5336006E5DB
:092AA100346002D322123137C364
:012AAA002209
:042214008F2A8D2B55
:10221800753005753105C203786A76C0AE02AF0322
:102228007C007D641212F8786BA607AE2EAF2F7C67
:10223800007D641212F8786CEFF6796AE718262F99
:10224800786DF6200345E5316041E52AC313452B37
:10225800FF7B007A00796A754404D20912269140FE
:1022680011E530600DD2087F0A7E00123066153005
:1022780080D87F907E0112316720F904D20380074D
:102288007F327E00120003153180B87F647E001211
:102298000003E5306006E5316002D322123137C30E
:0122A8002213
:0428AB008F2A8D2BB8
:1028AF00752F05753005C203786A76B008A603E563
:1028BF002DC313E52E13FF08F6796AE718262F7834
:1028CF006DF6200345E5306041E52AC313452BFF24
:1028DF007B007A00796A754404D20912269140115F
:1028EF00E52F600DD2087F0A7E00123066152F800B
:1028FF00D87F907E0112316720F904D20380077FC1
:10290F00327E00120003153080B87F647E00120003
:0F291F0003E52F6006E5306002D322123137C383
:01292E002286
:042AAB008F2A8D2BB6
:102AAF00752E05752F05C203786A76D008A6030820
:102ABF00A62D796AE71826252D786DF6200345E5B2
:102ACF002F6041E52AC313452BFF7B007A00796AFB
:102ADF00754404D2091226914011E52E600DD208DB
:102AEF007F0A7E00123066152E80D87F907E0112ED
:102AFF00316720F904D20380077F327E0012000372
:102B0F00152F80B87F647E00120003E52E6006E566
:092B1F002F6002D322123137C3EA
:012B2800228A
:04292F008F2A8D2B33
:10293300752C05752D05C203786A76E0EA08F6AFB3
:1029430003EB08F6796AE718262F786DF62003451E
:10295300E52D6041E52AC313452BFF7B007A0079FF
:102963006A754404D2091226914011E52C600DD2F8
:10297300087F0A7E00123066152C80D87F907E0176
:1029830012316720F904D20380077F327E001200E0
:1029930003152D80B87F647E00120003E52C6006CA
:0A29A300E52D6002D322123137C384
:0129AD002207
:0429AE008F2F8D30AA
:1029B200753105753205C205786A7620300404E661
:1029C2004401F6786B76AA0876BB796AE718262462
:1029D200BB786DF6200545E5326041E52FC313450E
:1029E20030FF7B007A00796A754404D2091226917D
:1029F2004011E531600DD2087F0A7E001230661563
:102A02003180D87F907E0112316720F904D205808F
:102A1200077F327E00120003153280B8E53160066E
:0A2A2200E5326002D322123137C3FF
:012A2C002287
:08245F008F348D358A368B376E
:10246700753A05753B05C205D3E5379539E53695C8
:10247700384006853836853937786A7638E536083C
:10248700F6AF37E53708F6FF796AE718262F786D34
:10249700F6200545E53B6041E534C3134535FF7B31
:1024A700007A00796A754404D2091226914011E531
:1024B7003A600DD2087F0A7E00123066153A80D83E
:1024C7007F907E0112316720F904D20580077F32A1
:1024D7007E00120003153B80B8E53B6005AE36AFC2
:0524E70037221231371D
:0124EC0022CD
:0419CA008F2E8D2FA0
:1019CE00753605753705C207E5332BE5323AC394F4
:1019DE00005009C3E49BF533E49AF532E5332BFF4F
:1019EE00E5323AFED3EF9535EE9534400AE5359B58
:1019FE00F533E5349AF532D3E5339400E53264805D
:101A0E0094804008786A7611D2068006786A76103D
:101A1E00C206300506786AE64404F6AF33AE3212DB
:101A2E0032D58E328F33E53345327003021AC0E55C
:101A3E0032FF3395E0EF786BF6AF33E53308F6FF00
:101A4E00796AE718262F786DF6200745E53760414D
:101A5E00E52EC313452FFF7B007A00796A75440487
:101A6E00D2091226914011E536600DD2087F0A7E0A
:101A7E0000123066153680D87F907E0112316720B5
:101A8E00F904D20780077F327E00120003153780DB
:101A9E00B8E53760197F037E00120003300605AEED
:101AAE0032AF3322C3E49533FFE49532FE22123176
:061ABE0037227E007F00CC
:011AC40022FF
:10188800300450AD5FAC5E7F1012302DAD5B7F230E
:10189800123106AD547F20123106AD557F24123126
:1018A80006AD567F25123106AD577F22123106AD9F
:1018B8005C7F26123106AD587F27123106AD5D7F59
:1018C80029123106AD5A7F28123106AD597F2112EF
:1018D8003106227F10122D638E5E8F5FC3E55F9401
:1018E80001E55E9400400BD3E55F94FCE55E94014E
:1018F8004006755E00755F017F231231BC8F5BD394
:10190800E55B648094845009C3E55B6480948050EF
:1019180003E4F55B7F201231BC8F54E554D3940A5D
:101928005007E554C39401500375540A7F241231BB
:10193800BC8F55E555D394965007E555C39401508F
:101948000375550A7F251231BC8F56E556D3943C52
:101958005007E556C3940150037556057F2612318A
:10196800BC8F5CD3E55C648094855009C3E55C64F6
:101978008094815003755C027F271231BC8F58E533
:1019880058D394645007E558C394015003755850D0
:101998007F291231BC8F5DD3E55D6480948A50093C
:1019A800C3E55D648094765003E4F55D7F281231C9
:1019B800BC8F5A7F211231BC8F597F221231BC8FC4
:0219C8005722A4
:0B331F0075988075A910C298C2992211
:10309E0053D8F8EF540742D8C2DBE4F52A75DA802C
:1030AE0020DCFD746A252AF8A6D97F037E00120063
:1030BE0003052AE52AC3940340E37F6A7D03122F9A
:0530CE00F3786BE6FF42
:0130D30022DA
:10326A00D291EF25E054074401786AF608A6057F53
:0B327A006A7D02122EAAC291D291229E
:041D6F008F348D35EB
:101D73007F541232B07BFF7A0779D7120E76E5349F
:101D8300601FFF3395E0FE7C007D0E1212917C6391
:101D93007D9CCFCDCFCECCCE1212F88E368F37802E
:101DA3000675366375379CE535249B604D046003E7
:101DB300021E44E4F538F539AE38AF397C007D6452
:101DC3001212F8AD07E4FF12326A7F477E00120059
:101DD30003E5372539F539E5363538F538C3E539BF
:101DE300949CE538648094E340CE7DFFE4FF123297
:101DF3006A7D147F041230D4C32275386375399C0D
:101E0300AE38AF397C007D641212F8AD07E4FF12DF
:101E1300326A7F477E00120003C3E5399537F539EF
:101E2300E5389536F538D3E5399400E53864809480
:101E33008050CDE4FDFF12326A7D147F041230D44A
:011E4300D3CB
:011E4400227B
:101C95007F541232B07BFF7A0779EC120E767532DB
:101CA5003CE4FBFD7FB0122A2D30B229C204E4FDCD
:101CB5007FB01229AE752D4E752E2030B217E52E48
:101CC500452D60117F017E00120003E52E152E7053
:101CD50002152D80E6D204E4FD7FB01229AE752DE4
:101CE5004E752E2020B217E52E452D60117F017E01
:101CF50000120003E52E152E7002152D80E6C2F8A0
:101D05007F017E00120003D2F87F647E001200037B
:101D15007538577539087B037A00E4FD7FB01224C6
:101D25005F7FFA7E00120003E55825E02419F5329D
:101D3500E4FBFD7FB0122A2DD2127B057A00E4FD6B
:101D45007FB012233EC211E52E452D70157F54122A
:101D550032B07BFF7A087901120E767F12122EF4CB
:091D650080FE7D147F041230D4CD
:011D6E002252
:102F3C007532A0E4FBFD7FB0122A2D752D00752E85
:102F4C00FA7B24E4FD7FB01228AB752E05752F1487
:102F5C007B587A02E4FD7FB0122214E4F52D7B64D9
:102F6C00FD7FB0122AAB7BA47A56E4FD7FB0122908
:022F7C002F2202
:102606007BFF7A087914120E767F401232B07BFF78
:102616007A087924120E7620B25A7BA47A56E4FD03
:102626007FB012233EC204E4FD7FB01229AE7FE8DC
:102636007E03120003752A4E752B2020B217E52B58
:10264600452A60117F057E00120003E52B152B70CD
:1026560002152A80E6C2F87F017E00120003D2F836
:10266600E52B452A700E7F10122EF47BFF7A08792F
:1026760037122FB97F141232B07BFF7A08794912CC
:0A2686000E76121C951232857F01BA
:012690002227
:02217A008F34A0
:10217C001534E534700302220F25E02440FF122DA4
:10218C00638E358F36E53425E025E024B2F582E404
:10219C00340BF58312133FEF241EFBE43EFAE43DAF
:1021AC00F9E43CF8AE35AF36E4FCFDC312132E4017
:1021BC002FE53425E025E024B2F582E4340BF583D9
:1021CC0012133FEF24E2FBEE34FFFAED34FFF9EC8F
:1021DC0034FFF8AE35AF36E4FCFDD312132E401E9F
:1021EC007D037C007FC87E0012203EE53425E0256F
:1021FC00E024B2F582E4340BF58312133F22AE35A2
:07220C00AF36227E007F00C7
:0122130022A8
:0613DE008F2D8C2E8D2FD7
:1013E400852D30753105E562B52D01227F14123249
:1013F400B0E52F452E600DE55760097D65AF5612A7
:101404001D6F9217E52DB4011AE554C3132401FF8F
:10141400E433FED3E5629FEE6480F8748098400361
:10142400752D0B75310520FF03021573E52DD3953A
:1014340054405C7BFF7A08795D120E763012277F68
:101444000B12217AAD5DED3395E0FCEF2DFFEE3C00
:10145400CF2405FBE43FFA753857753908E4FD7F5E
:10146400B012245F801F7F0B12217AAD5DED33959E
:10147400E0FCEF2DFBEE3CFA753857753908E4FDB6
:101484007FB012245FB211D212753001021563E5E8
:101494002DC3940150673012157F0B12217AEF246B
:1014A40005FBE43EFAE4FD7FB012233E80107F0B7F
:1014B40012217AAA06AB07E4FD7FB012233E7BFF1C
:1014C4007A087972120E76E55BB4030FE55CB40416
:1014D4000AE55420E00514F52D800385542DAF2D25
:1014E40012217AAA06AB077538567539A4E4FD7F34
:1014F400B012245FB211C212852D308062E52DD363
:1015040095624030AF2D12217A8E328F33EF24054D
:10151400FBE43EFA7538567539A4E4FD7FB0122415
:101524005FD2127BFF7A08798785323F8533401278
:101534000E76802BAF2D12217AAA068A32AB078B46
:10154400337538567539A4E4FD7FB012245FC21296
:101554007BFF7A08799A85323F853340120E767F75
:10156400647E001200031531E531600302142AE59C
:101574003170157F541232B07BFF7A0879AD120EA8
:0C158400767F11122EF480FED216AF30DC
:011590002238
:03004B0002333449
:05333400D213C2B93202
:03002300022C9715
:102C9700C0E0C0D075D008309A41301556301418AE
:102CA700C214E59960057563018048756302E561A3
:102CB700156170021560803BE5614560600AE5615A
:102CC700156170021560802B74652564F8A699E577
:102CD7006460041564801CC2158018E599700F851F
:102CE7005E60855F61756404D214D2158005C215D4
:0A2CF70075630AC298D0D0D0E03215
:101E4500855B2BC203D205A2039206122E5FEF64B7
:101E550002607BBF040E155BC3E55B648094805014
:101E650003E4F55BBF080E055BD3E55B64809484F2
:101E75004003755B04EF640170287F541232B07B18
:101E8500FF7A0879B9120E76D2041218887FE87E97
:101E9500031200037F541232B07BFF7A0879C31214
:101EA5000E767F401232B0AF5BEF3395E0FE7C00DB
:101EB5007D1412129174DE2FF9740B3EFA7BFF121A
:101EC5000E76E55924FF9203123305021E4AE52BCF
:101ED500B40408E55B6404600280FEE52B640360DE
:101EE50010E55BB4030B7D017C007F011213DE8FCF
:011EF500628A
:011EF60022C9
:101EF700C205C206122E5FEF64027003021F90BF75
:101F07000417055FE55F7002055ED394FCE55E94F8
:101F1700014006755E00755F01BF0819E55F155F33
:101F27007002155EC3E55F9401E55E940050067587
:101F37005E01755FFCEF640170287F541232B07B3D
:101F4700FF7A0879B9120E76D2041218887FE87ED4
:101F5700031200037F541232B07BFF7A0879C31251
:101F67000E767F401232B07BFF7A0879CD855E3FCF
:101F7700855F40855E41855F42120E767FC87E0091
:101F8700120003123305021EF7E55924FF92087F5A
:061F97000A7E0012306614
:011F9D002221
:1023CF0085542BC205C206122E5FEF6402606BBFED
:1023DF00040C0554E554D3940A400375540ABF08FE
:1023EF000C1554E554C394015003755401EF640167
:1023FF0070287F541232B07BFF7A0879B9120E76AB
:10240F00D2041218887FE87E031200037F54123221
:10241F00B07BFF7A0879C3120E767F401232B07B01
:10242F00FF7A0879E2753F00855440120E767FC817
:10243F007E001200031233058089E55924FF9208AC
:0F244F007F0A7E00123066E554652B600280FE26
:01245E00225B
:1027A100C205C206122E5FEF6402606BBF040C0506
:1027B10055E555D394964003755501BF080C155541
:1027C100E555C394015003755596EF640170287F58
:1027D100541232B07BFF7A0879B9120E76D2041204
:1027E10018887FE87E031200037F541232B07BFF0A
:1027F1007A0879C3120E767F401232B07BFF7A08D5
:1028010079F4753F00855540120E767FC87E00121F
:1028110000031233058089E55924FF92087F0A7E5F
:04282100001230660B
:012825002290
:10282600C205C206122E5FEF6402606BBF040C0580
:1028360056E556D3943C4003755601BF080C155611
:10284600E556C39401500375563CEF640170287F2A
:10285600541232B07BFF7A0879B9120E76D204127E
:1028660018887FE87E031200037F541232B07BFF84
:102876007A0879C3120E767F401232B07BFF7A094E
:102886007903753F00855640120E767FC87E00128A
:1028960000031233058089E55924FF92087F0A7EDA
:0428A6000012306686
:0128AA00220B
:102B2900C203D205A2039206122E5FEF6402606906
:102B3900EF64046003BF080CE55770047E0180024E
:102B49007E008E57EF640170287F541232B07BFFEC
:102B59007A0879B9120E76D2041218887FE87E03B2
:102B69001200037F541232B07BFF7A0879C3120E28
:102B7900767F401232B0E557600B7BFF7A097912F4
:102B8900120E7680097BFF7A09791C120E76E559B7
:092B990024FF9203123305808928
:012BA2002210
:101F9E00855C2BC203D205A2039206122E5FEF645C
:101FAE0002607BBF040E155CC3E55C6480948150B7
:101FBE0003755C01BF080E055CD3E55C64809485F7
:101FCE004003755C05EF640170287F541232B07BBC
:101FDE00FF7A0879B9120E76D2041218887FE87E3D
:101FEE00031200037F541232B07BFF7A0879C312BA
:101FFE000E767F401232B0AF5CEF3395E0FE7C0080
:10200E007D1212129174302FF9740C3EFA7BFF126E
:10201E000E76E55924FF9203123305021FA3E52B1A
:0F202E00655C600B7D017C007F011213DE8F6209
:01203D002280
:1022A900C205C206122E5FEF6402606BBF040C0503
:1022B90058E558D394644003755801BF080C155864
:1022C900E558C394015003755864EF640170287F81
:1022D900541232B07BFF7A0879B9120E76D2041201
:1022E90018887FE87E031200037F541232B07BFF07
:1022F9007A0879C3120E767F401232B07BFF7A09D1
:102309007926753F00855840120E767FC87E0012E7
:1023190000031233058089E55825E02419F532E4D4
:10232900FBFD7FB0122A2DE55924FF92087F0A7E12
:0423390000123066F8
:01233D00227D
:102BA300C203D205A2039206122E5FEF640260698C
:102BB300EF64046003BF080CE55A70047E018002D1
:102BC3007E008E5AEF640170287F541232B07BFF6F
:102BD3007A0879B9120E76D2041218887FE87E0338
:102BE3001200037F541232B07BFF7A0879C3120EAE
:102BF300767F401232B0E55A600B7BFF7A09793851
:102C0300120E7680097BFF7A097943120E76E55915
:092C130024FF92031233058089AD
:012C1C002295
:102E1300C2037D147F041230D4D205A2039206129A
:102E23002E5F8F2BEF6402602B7F401232B07F3016
:102E33001231BC753F008F407BFF7A09794E120E29
:102E4300767F141232B0122DBDE55924FF9203127E
:0B2E5300330580C57D147F031230D4CE
:012E5E002251
:102C1D00C203D205A2039206122E5FEF6402606911
:102C2D00EF64046003BF080CE55970047E01800257
:102C3D007E008E59EF640170287F541232B07BFFF5
:102C4D007A0879B9120E76D2041218887FE87E03BD
:102C5D001200037F541232B07BFF7A0879C3120E33
:102C6D00767F401232B0E559600B7BFF7A097912FD
:102C7D00120E7680097BFF7A09791C120E76E559C2
:092C8D0024FF9203123305808933
:012C9600221B
:101AC500C2037F401232B07BFF7A09795C120E7631
:101AD500E55924FF9203123305D205A2039206129B
:101AE5002E5FEF64016003021BB0F55BF55E755F69
:101AF5000175540A75550A755605F557755C0275D5
:101B05005850755A017559011232307F541232B04E
:101B15007BFF7A097970120E76D2041218887FE855
:101B25007E031200037D147F041230D47F401232ED
:101B3500B07BFF7A09797C120E76123305D205A2A5
:101B4500039206122E5FEF64017060F52BD3E52B2F
:101B55006480948A4003D38001C34033E52B25E09C
:101B65002440FFC007AF2BEF3395E0FEEF7802C3AB
:101B750033CE33CED8F924B2F582740B3EF58312F9
:101B8500133FAD07AC06D00712302D052B80BE7F65
:101B9500541232B07BFF7A097991120E767FE87E76
:0B1BA500031200037D147F041230D4F3
:011BB0002212
:10159100C203C204E5626401600302170DD205A211
:1015A100039206122E5F8F2BEF6402700302172243
:1015B100E562640A7003021722E52B6401600302ED
:1015C10016F37F401232B07BFF7A09799D120E76B5
:1015D100755850E55825E02419F532E4FBFD7FB03C
:1015E100122A2D756202E562D3940A4003D3800169
:1015F100C350030216F1E56225E025E024AEF58231
:10160100E4340BF58312133FEF24E7FBEE34FFFACA
:101611007538567539A4E4FD7FB012245F7FFA7ED8
:1016210000120003752DC220FF0A7F327E001200D6
:1016310003D52DF3E52D700280FE752CE27F541247
:1016410032B07BFF7A0979AE753F00856240AF2CDD
:10165100EF3395E0F5418F42120E76123305D20534
:10166100A2039206122E5F8F2BE52B6404702D05C9
:101671002CF5327533017534567535A4C205FBFA64
:10168100FD7FB01219CA752DC220FF0A7F0A7E00A4
:10169100120003D52DF3E52D700280FEC3E52C6405
:1016A10080949E5006E52B640170927F541232B0F3
:1016B1007BFF7A0979C4120E76E56225E025E024E4
:1016C100AEF582E4340BF58312133FAD2CED339567
:1016D100E0FCEF2DFDEE3CFCE56214FF25E024402B
:1016E100FF12302D7FE87E0312000305620215E729
:1016F10080FE7F401232B07BFF7A0979D9120E76D3
:10170100E55924FF920312330502159E7F401232E0
:10171100B07BFF7A0979EA120E767FE87E03120028
:0117210003C4
:0117220022A4
:1024ED00C205C206122E5FEF64026073BF040E05B3
:1024FD005DD3E55D6480948A4003755D0ABF080E67
:10250D00155DC3E55D648094765003755DF6EF64EB
:10251D000170287F541232B07BFF7A0879B9120E00
:10252D0076D2041218887FE87E031200037F5412BE
:10253D0032B07BFF7A0879C3120E767F401232B02B
:10254D007BFF7A0979FDAF5DEF3395E0F53F8F4065
:10255D00120E767FC87E001200031233058081E5CE
:0C256D005924FF92087F0A7E001230669D
:01257900223F
:101BB100C2037F401232B07BFF7A0A7914120E768B
:101BC100123305D205D206122E5FEF6401600302C3
:101BD1001C947F401232B0E4FD7FB012271A400DF1
:101BE1007BFF7A0A7926120E76D20380097BFF7A6F
:101BF1000A7938120E767FD07E071200037532A063
:101C0100E4FBFD7FB0122A2DE4FDFC7F011213DEFF
:101C11008F627FDC7E05120003752B0B752CB820BB
:101C2100FF1A7F0A7E00120003E52C152C700215A5
:101C31002BD3E52C9400E52B940050E37D147F0316
:101C41001230D47F401232B0E52C452B600B7BFF64
:101C51007A0A794A120E76800B7BFF7A0A795C1236
:101C61000E76D2037FD07E0712000320030E121CD2
:101C7100957BFF7A0A796E120E7680097BFF7A0ACC
:101C81007984120E767F401232B07F887E13120063
:031C91000380FECF
:011C9400222D
:10319200123285E4FF1232B07BFF7A0A799A120E5C
:1031A200767F401232B07BFF7A0A79A9120E76122C
:0A31B20031E37FF0122EF480FE22BC
:10172300E4F52A123285E4FF1232B0AF2AEF339583
:10173300E0FE7C007D12121291749C2FF9740C3E12
:10174300FA7BFF120E767F541232B07BFF7A0A794E
:10175300BA120E761231E3123305D205E55924FF8E
:101763009206122E5FEF64027003021880BF040A10
:10177300052AE52AB40F03E4F52ABF080E152AC388
:10178300E52A648094805003752A0EEF6401600398
:1017930002185A7F541232B07BFF7A0A79CF120EA5
:1017A30076E52AB40F00400302182D9017B5F828E8
:1017B30028730217E20217E70217EC0217F1021768
:1017C300F60217FB02180002180502180A02180F86
:1017D30002181402181902181E02182302182812DC
:1017E3001E45805B121EF780561223CF80511227AD
:1017F300A1804C1228268047121F9E8042122B295B
:10180300803D1222A98038122BA38033122C1D8015
:101813002E121AC5802912159180241224ED801FDF
:10182300122E13801A121BB180157F401232B07B27
:10183300FF7A0A79DB120E767FE87E031200037DBE
:10184300147F021230D47F541232B07BFF7A0A79AC
:10185300ED120E761231E3E4FF1232B0AF2AEF330A
:1018630095E0FE7C007D12121291749C2FF9740C8A
:101873003EFA7BFF120E7612330502175D7D147F4D
:04188300041230D447
:01188700223E
:10004E00E4F5237524FA75251E7526FFD200D2011C
:10005E00D202F587F5D012332A12332F12331FD264
:10006E00BED297F563C2041218887E007F007D050C
:10007E007B007A00796512134FD2B9C2CDD2AFD2BE
:10008E009CC298D2ACD203122D01E4FF1232B07B87
:10009E00FF7A0A79F9120E767F471232B07BFF7A19
:1000AE000B790E120E767F591232B07BFF7A0B79D6
:1000BE001B120E76D2031232E77FB87E0B120003AC
:1000CE001232857E007F067D007B007A00797412E5
:1000DE00134FE4F527E4FDAF2712326A7F0A7E0044
:1000EE001200030527E527C3940240E9E4FD7FB023
:1000FE0012271A40097BFF7A0B792B122FB9D208DF
:10010E007FC87E00123066122F3CC205C206122E28
:10011E005FEF6403703F7F401232B07BFF7A0B7942
:10012E003C120E76E4F527D2087F647E001230660C
:10013E007F647E001200030527E527C3940A40E77B
:10014E00E4FBFAFD7FB012233E7562017D147F023F
:10015E001230D480051226068F62E55575F00AA47A
:10016E0085F028F529E55BB403077DFFE4FF123225
:10017E006AE52660041526800B7526FFE4F525C278
:10018E0003122D01E4FF1232B0AF5BEF3395E0FEA8
:10019E007C007D0912129174AA2FF9740D3E753FE1
:1001AE00FFF54089417BFF7A0B794A7542008562E3
:1001BE0043754400855445120E7620130320943760
:1001CE00D2031232E77524FAC205C206122E5F8FD1
:1001DE0023BF030ED297D2087F0A7E00123066121A
:1001EE003192E523B40113D297D2087F0A7E001212
:1001FE0030661217238003E4F523E4F527E527750F
:10020E00F003A42474FFC3740495272465F8E6FB59
:10021E007D0312324EE52775F003A42474F9E4FA37
:10022E00FB786A7C00FDFE7F031212407F6A7D031D
:10023E00122FF3786BE6FF74152527F8A60705270E
:10024E00E527C3940240B6E5256004152580287F76
:10025E005A1232B0E56375F00FA424D7F9740D3538
:10026E00F0753FFFF54089417BFF7A0779A3120EA7
:10027E007675251EE4F563E4FF12309E7813A6070B
:10028E007F0112309E7814A607E55B602724FC6080
:10029E00630470707F401232B0AE28AF297C007DAF
:1002AE000A1212A38E3F8F407BFF7A0B795C120EDF
:1002BE00760203527F401232B07813E6FF7E007C46
:1002CE00007D641212917DFF1212A3AA06AB07786D
:1002DE0014E6FF7E007C007D641212917DFF1212E7
:1002EE00A38E418F428A3F8B407BFF7A0B7971122E
:1002FE000E7680507F401232B07BFF7A0B798A12D5
:10030E000E7680407F401232B0AF697E007C007D59
:10031E00641212917DFF1212A3AA06AB07AF687E7C
:10032E00007C007D641212917DFF1212A38E438F0A
:10033E00448A418B427BFF7A0B799A855E3F855FBB
:10034E0040120E76E55B14700302048714700302EC
:10035E0005341470030205BD14700302070D240446
:10036E00600302071D7813E6FFD3943F4013EF940A
:10037E0066500E08E6FF943F4007EF94665002C2A7
:10038E000030160302071DE52324F8601724FC60D5
:10039E002224087029E56204FF7D017C001213DE21
:1003AE008F62801AE56214FF7D017C001213DE8FCE
:1003BE0062800B7D017C007F011213DE8F623000A4
:1003CE000302071D7813E6C39434501508E6943FD4
:1003DE00400FE56204FF7D017C001213DE8F62D2B6
:1003EE00007813E6D3943F401508E69434500FE599
:1003FE006214FF7D017C001213DE8F62D20078132F
:10040E00E6C39434501408E6C39434500D7D017C39
:10041E00007F011213DE8F62D2007813E6D394B4FC
:10042E00401508E69466500FE56204FF7D017C00DE
:10043E001213DE8F62D2007813E6C394665015084D
:10044E00E694B4400FE56214FF7D017C001213DECA
:10045E008F62D2007813E6D394B4500302071D08BE
:10046E00E6D394B4500302071D7D017C007F011278
:10047E0013DE8F62D20002071D7815E6C3944C502E
:10048E000908E6C3944C5002C20130160302071D40
:10049E00E52324F8601624FC602024087026E5620B
:1004AE0004FFE4FDFC1213DE8F628018E56214FF78
:1004BE00E4FDFC1213DE8F62800AE4FDFC7F011264
:1004CE0013DE8F6230010302071D7815E6D394B355
:1004DE00401408E6944C500EE56204FFE4FDFC1255
:1004EE0013DE8F62D2017815E6C3944C501408E6E1
:1004FE0094B3400EE56214FFE4FDFC1213DE8F622E
:10050E00D2017815E6D394B3500302071D08E6D343
:10051E0094B3500302071DE4FDFC7F011213DE8F1E
:10052E0062D20102071D7816E6C3944C5002C20136
:10053E0030160302071DE52324F8601624FC602004
:10054E0024087026E56204FFE4FDFC1213DE8F62C0
:10055E008018E56214FFE4FDFC1213DE8F62800A40
:10056E00E4FDFC7F011213DE8F6230010302071DD2
:10057E007816E6D394B3500302071D18E6D39406FB
:10058E00500302071D752701E527900E0393FF7890
:10059E0015E6D39F400AE52795545004052780E8B9
:1005AE00E4FDFCAF271213DE8F62D20102071D306D
:1005BE00160302071DE52324F8601724FC6022248D
:1005CE00087029E56204FF7D017C001213DE8F6244
:1005DE00801AE56214FF7D017C001213DE8F6280AB
:1005EE000B7D017C007F011213DE8F62E529452809
:1005FE006003020703E55C24FE602C14604D14605A
:10060E007A1470030206BF240460030206F6E56244
:10061E00655470030206F6E56204FF7D017C00124C
:10062E0013DE8F620206F6E55A6010E56204FF7D66
:10063E00017C001213DE8F620206F6E56214FF7D66
:10064E00017C001213DE8F620206F630020FE562A5
:10065E0004FF7D017C001213DE8F62800DE56214B3
:10066E00FF7D017C001213DE8F62E562B55402C27B
:10067E0002E56264017071D202806DE55A6010E588
:10068E00622402FF7D017C001213DE8F628059E529
:10069E0062B4010D7D017C00E4FF1213DE8F6280D7
:1006AE0047E56224FEFF7D017C001213DE8F62801F
:1006BE0037300210E5622402FF7D017C001213DE4A
:1006CE008F62800EE56224FEFF7D017C001213DE38
:1006DE008F62E55424FEFFE562D39F4002C202E51D
:1006EE0062C394025002D202E55575F00AA485F059
:1006FE0028F529801AE5291529700215288010750C
:10070E006201E55A24FF9204E4FD7FB01229AEE5A2
:10071E005B64036004E55B70097F0A7E00120003D0
:10072E00801BE4F527C3740295272465F8E6FDAF18
:10073E002712326A0527E527C3940240E830163B9C
:10074E0030FF38E5626401701D30120B7B05FAFD37
:10075E007FB012233E8009E4FBFAFD7FB012233EE8
:10076E00301103121C95C2163017097D64AF561254
:10077E001D6F92177D147F031230D4E5246004158B
:0D078E00248005C2031232E7C29702017FEA
:01079B00223B
:10000300E4FDEF4E6018EF1F70011E7C66EC600884
:0E0013001CEDF5F0A4FD80F5D2AED2BE80E467
:0100210022BC
:10316700AD07AC06ED7803CEC313CE13D8F9FDAC8B
:10317700067802CEC313CE13D8F92DFDEE3CFCED35
:0B3187004C6007ED1D70F81C80F52265
:02004800002294
:103066008E3F8F40300830D2ECC2EEE54025E0F5C9
:1030760040E53F33F53FE540453F6017E5401540E5
:103086007002153F7FF47E01123167B2EBD2AED2E9
:08309600BE80E3C2ECC2EB2294
:10203E008E378F388C398D3AE5397056E53A146003
:10204E002314603314603824037047753927753AAA
:10205E0010E538AE377802CEC313CE13D8F9F53863
:10206E008E378045753913753A88E537C313F537C2
:10207E00E53813F5388032753909753AC4802A75FA
:10208E003903753AE8E53825E0F538E53733F537A5
:10209E008017753901753AF4E538AE377802C333D7
:1020AE00CE33CED8F9F5388E37D2ECC2EEE53845C0
:1020BE00376017E538153870021537AF3AAE39125A
:0F20CE003167B2EBD2AED2BE80E3C2ECC2EB22DE
:0433390000401454E8
:0D331200D2EDD2EDC2ED7F147E00023167D6
:102F7E007552FF85E85343E80FC2ECC2EFD2EED292
:102F8E00ED7F287E0012316730EB13E552600F158E
:102F9E00527F147E00123167D2AED2BE80EAC2EDED
:0A2FAE008553E8E5526002D322C308
:012FB80022F6
:100026008F51C2EC122F7E53E8F0E551C4540F54A1
:100036000F42E812331253E8F0E551540F42E8023A
:02004600331273
:1032B0008F3CC2EC122F7EC2EFC2EEE53C4480FF91
:0332C000020026E3
:10329B008F12C2EC122F7EC2EFC2EEE512444054E5
:0532AB007FFF02002678
:102D0100E4F5E83003087F14FE12000380077F0119
:102D11007E0012000375E8031233127F057E001254
:102D21000003122D56122D5675E8021233127F013F
:102D31007E001200037F281200267F0C1200267FDE
:102D4100061200267F011200267F021200267F0252
:102D51007E0002000375E8031233127F017E000238
:022D610000036D
:103285007F011200267F027E001200037F021200DA
:0632950026E4FF0232B046
:0E32F7008F50D2EFC2EE120026C2EFAF50226F
:1030D4008F3A8D3B1230F1E53B600D153B7F20129A
:1030E40032F7D2AED2BE80EFAF3A0230F1EF339571
:1030F400E0FE74382FF58274333EF583E493FF02C7
:0231040032B0E7
:1032E700300304C2968002D2967F017E000200035B
:10324E00ED14FEEED39400400EEF2E14F8E6FDEFD3
:0B325E002EF8A6051E80ECA807A603B2
:013269002242
:02320A00A80713
:10320C00E4F510F511FFEFC39D500EE62511F511F5
:10321C00E43510F5100F0880EDED7C00AE10AF1109
:03322C001212F883
:01322F00227C
:102FF300ED14FEC3EE64809480402E7D01D3EE6415
:1030030080F8ED648098501EEF2DF8E6FCE814F884
:10301300E6FBD39C400DA903EF2D14F8A604EF2D76
:09302300F8A6010D80D71E80CA39
:01302C002281
:0300000002257A5C
:0C257A00787FE4F6D8FD7581790225C158
:10117000E709F608DFFA8046E709F208DFFA803E61
:1011800088828C83E709F0A3DFFA8032E309F6084E
:10119000DFFA8078E309F208DFFA807088828C83B6
:1011A000E309F0A3DFFA806489828A83E0A3F6086A
:1011B000DFFA805889828A83E0A3F208DFFA804C44
:1011C00080D280FA80C680D4806980F2803380101B
:1011D00080A680EA809A80A880DA80E280CA803384
:1011E00089828A83ECFAE493A3C8C582C8CCC583FC
:1011F000CCF0A3C8C582C8CCC583CCDFE9DEE780CC
:101200000D89828A83E493A3F608DFF9ECFAA9F04A
:10121000EDFB2289828A83ECFAE0A3C8C582C8CCA0
:10122000C583CCF0A3C8C582C8CCC583CCDFEADEB9
:10123000E880DB89828A83E493A3F208DFF980CC1B
:1012400088F0EF60010E4E60C388F0ED2402B40414
:101250000050B9F582EB2402B4040050AF232345BB
:0612600082239011C0730F
:10126600BB010689828A83E0225002E722BBFE0286
:09127600E32289828A83E49322B9
:10127F00BB010689828A83F0225002F722BBFE014E
:02128F00F32248
:10129100EF8DF0A4A8F0CF8CF0A428CE8DF0A42E71
:0212A100FE222B
:1012A300BC000BBE0029EF8DF084FFADF022E4CC2F
:1012B300F875F008EF2FFFEE33FEEC33FCEE9DECF8
:1012C300984005FCEE9DFE0FD5F0E9E4CEFD22ED3E
:1012D300F8F5F0EE8420D21CFEADF075F008EF2F88
:1012E300FFED33FD4007985006D5F0F222C398FD79
:0512F3000FD5F0EA2216
:1012F800C2D5EC30E709B2D5E4C39DFDE49CFCEE11
:1013080030E715B2D5E4C39FFFE49EFE1212A3C3D3
:10131800E49DFDE49CFC80031212A330D507C3E4CE
:061328009FFFE49EFE227F
:10132E00EB9FF5F0EA9E42F0E99D42F0E89C45F015
:01133E00228C
:10133F00E493FC740193FD740293FE740393FF22F4
:100E1400E54B243FF8E6054B22783C300F02783F3F
:100E2400E475F0011213A80212662008EB7F2ED29B
:100E3400088018EF540F2490D43440D4FF300C0BA6
:100E4400EF24BFB41A0050032461FFE54C6002157F
:100E54004C054FE54F7002054E300F0D783CE4759C
:100E6400F0011213A8EF02127F0232F77403D20FBB
:100E74008003E4C20FF54B8B3C8A3D893EE4F54C7C
:100E8400F54EF54FE54C60077F20120E4F80F57547
:100E94004DFFC209C208C20AC20BC20DC20EC21063
:100EA400120E1DFF700D300F057F00120E60AF4F44
:100EB400AE4E22B4255FC2D5C20C120E1DFF24D043
:100EC400B40A00501A75F00A784C30D50508B6FFFC
:100ED4000106C6A426F620D5047002D20B80D924BC
:100EE400CFB41A00EF5004C2E5D20C021060D2094C
:100EF40080C6D20880C0D20A80BCD2D580BAD20DB6
:100F040080B47F20120E4F200A077401B54C0040B4
:100F1400F1120E14FF120E4F020E88D210D20E8060
:100F240095120E14FB120E14FA120E14F94A4B7099
:100F34000679317A117BFF200A2EE54C602A7E0067
:100F44008E8275830012137B60060EEE654D70F081
:100F5400C2D5EBC0E0EAC0E0E9C0E0EE1210A7D0D1
:100F6400E0F9D0E0FAD0E0FB121266FF60AAEBC011
:100F7400E0EAC0E0E9C0E0120E4FD0E02401F9D06D
:100F8400E03400FAD0E0FBE54D0460DCD54DD980B7
:100F9400877BFF7A1079A3D20A809C79108002792A
:100FA40008C20EC2108008D2D5790A8004790AC218
:100FB400D5E54D047002F54DE4FAFDFEFF120E1462
:100FC400FC7B08200913120E14FD7B1030080A1252
:100FD4000E14FE120E14FF7B20EC3382D592D550F2
:100FE40013C3E43008069FFFE49EFEE42009039D3A
:100FF400FDE49CFCE4CBF8C209EC700CCFCECDCC64
:10100400E824F8F870F38017C3EF33FFEE33FEEDF6
:1010140033FDEC33FCEB33FB994002FB0FD8E9EBD7
:10102400300905F8D0E0C448B209C0E00AEC4D4EDE
:101034004F78207B0070C2EAB54D0040BCC0E0127E
:1010440010A9D0F0D0E0200904C4C0E0C4B209C0A3
:10105400F0120E38D0F0D5F0EB020E881213B80F50
:1010640025530F9F580EF64C0EF2420FA34F0FABB1
:10107400440FAB490F0B430FB1550F95460F9545E0
:101084000F95471151500EFA2D0EFE2E0F212B0FE6
:1010940002230F1F20113F2A0EBA4800000F193FE8
:1010A4003F3F00790AA2D5200B14300D09B9100274
:1010B4000404B9080104A2D5200E02500104200A38
:0510C40068920AB54C22
:1010C900005034C0E07F20300B197F30A20A720E25
:1010D900720D500F121100C20AC20EC20DC2107F4A
:1010E90030800F300D03E9C0E0120E4F300D03D0F0
:1010F900E0F9D0E0B54CCC300D177F30B9100C12A7
:101109000E4F7F58300C077F788003B90803120E01
:101119004F300A057F2D020E4F7F202010F87F2BBC
:10112900200EF322920A80CF286E756C6C29002D4F
:1011390050434958D209120E143009F8C209784CA3
:1011490030D50108F6020EBA120E142403B40500B4
:101159004001E490113893120E40743A120E40D2B5
:071169000B754C04020F9FFF
:1032D500C3EE6480948040028007C3E49FFFE49EB0
:0232E500FE22C7
:10134F00EF4E6012EF60010EEDBB010B89828A83B5
:10135F00F0A3DFFCDEFA2289F05007F709DFFCA9C2
:0C136F00F022BBFEFCF309DFFCA9F02219
:1025860002004EE493A3F8E493A34003F68001F21D
:1025960008DFF48029E493A3F85407240CC8C33356
:1025A600C4540F4420C8834004F456800146F6DF25
:1025B600E4800B01020408102040809032C3E47EC0
:1025C600019360BCA3FF543F30E509541FFEE4931A
:1025D600A360010ECF54C025E060A840B8E493A3E1
:1025E600FAE493A3F8E493A3C8C582C8CAC583CA0C
:1025F600F0A3C8C582C8CAC583CADFE9DEE780BEC4
:0132D40000F9
:10137B00BB010CE58229F582E5833AF583E0225027
:10138B0006E92582F8E622BBFE06E92582F8E22271
:0D139B00E58229F582E5833AF583E493228B
:1013A800FAE6FB0808E6F925F0F618E6CA3AF62246
:1013B800D083D082F8E4937012740193700DA3A3C4
:1013C80093F8740193F5828883E4737402936860D8
:0613D800EFA3A3A380DFD8
:00000001FF
